:1000000019C035C034C033C032C031C030C02FC079
:100010002EC02DC02CC02BC02AC029C028C027C08C
:1000200026C025C024C023C022C021C089C01FC053
:100030001EC01DC011241FBECFEFCDBFDFE3DEBF4A
:100040001EE3A0E0BEE3E0E2FAE002C005900D92FC
:10005000AC33B107D9F72EE3ACE3BEE301C01D9288
:10006000A734B207E1F70E9459000C940E050C94D6
:100070000000E0E0F6E0808184608083818182601E
:100080008183828180618283828182838081816099
:1000900080830895E0E0F6E086838385816083872E
:1000A000808581608087838580FFFDCF80911006E9
:1000B00008956CE675E080E090E00E9487000E9461
:1000C00039007894C6E0DEE386E00E944A0080951D
:1000D00080933C3E1F928F93DF93CF930E94F90051
:1000E0009AE22CE28AE0915020408040E1F7000043
:1000F0000F900F900F900F90E7CFE0E0F8E0948121
:1001000095FFFDCF8093020880E090E00895E0E243
:10011000F4E0258124602583218124602183E0E0AF
:10012000F8E0608771878681806C8683858180682E
:10013000858360E070E08DE790E00E94AE00089556
:100140001F920F920FB60F9211248F938091000887
:100150008F910F900FBE0F901F9018950F931F93C4
:10016000CF93DF93009731F46115710519F480E0A6
:1001700090E03AC08B01EC016EE070E081E090E02D
:100180000E94E102FC01892B91F380E88383011531
:10019000110571F00287138781E8838380913D3ECA
:1001A00090913E3E892B21F4E0933D3EF0933E3EFC
:1001B0002097C9F0C087D187838182608383809133
:1001C0003F3E9091403E892B71F4E0933F3EF09387
:1001D000403E8091413E9091423E892B21F4E09334
:1001E000413EF093423ECF01DF91CF911F910F919D
:1001F0000895A0E0B0E0EFEFF0E00C94ED04AE0164
:100200004B5F5F4FFA0161917191AF0180913F3E69
:100210009091403E0E940F01E2E00C940605ACE094
:10022000B0E0E5E1F1E00C94DD047C016B018A01B2
:10023000FC0116821782838181FFBDC1CE01019628
:100240004C01F7019381F60193FD859193FF819114
:100250006F01882309F4ABC1853239F493FD859190
:1002600093FF81916F01853229F4B70190E00E94DC
:100270004704E7CF512C312C20E02032A0F48B3200
:1002800069F030F4803259F0833269F420612CC077
:100290008D3239F0803339F4216026C02260246029
:1002A00023C0286021C027FD27C030ED380F3A3029
:1002B00078F426FF06C0FAE05F9E300D1124532E1D
:1002C00013C08AE0389E300D1124332E20620CC0FA
:1002D0008E3221F426FD6BC1206406C08C3611F4E9
:1002E000206802C0883641F4F60193FD859193FFA2
:1002F00081916F018111C1CF982F9F7D95549330CB
:1003000028F40C5F1F4FFFE3F9830DC0833631F0F3
:10031000833771F0833509F05BC022C0F80180811A
:1003200089830E5F1F4F44244394512C540115C000
:100330003801F2E06F0E711CF801A080B18026FF39
:1003400003C0652D70E002C06FEF7FEFC5012C8701
:100350000E943C042C0183012C852F77222E17C08C
:100360003801F2E06F0E711CF801A080B18026FF09
:1003700003C0652D70E002C06FEF7FEFC5012C87D1
:100380000E942A042C012C852068222E830123FC44
:100390001BC0832D90E048165906B0F4B70180E2E7
:1003A00090E00E9447043A94F4CFF50127FC859130
:1003B00027FE81915F01B70190E00E944704311050
:1003C0003A94F1E04F1A51084114510471F7E5C015
:1003D000843611F0893639F5F80127FF07C06081AE
:1003E0007181828193810C5F1F4F08C06081718190
:1003F000072E000C880B990B0E5F1F4F2F76722E65
:1004000097FF09C090958095709561957F4F8F4FAC
:100410009F4F2068722E2AE030E0A4010E947F04E2
:10042000A82EA81844C0853729F42F7EB22E2AE0C2
:1004300030E025C0F22FF97FBF2E8F36C1F018F4BF
:10044000883579F0B4C0803719F0883721F0AFC013
:100450002F2F2061B22EB4FE0DC08B2D8460B82EDC
:1004600009C024FF0AC09F2F9660B92E06C028E05D
:1004700030E005C020E130E002C020E132E0F801C8
:10048000B7FE07C060817181828193810C5F1F4F2D
:1004900006C06081718180E090E00E5F1F4FA40173
:1004A0000E947F04A82EA818FB2DFF777F2E76FED2
:1004B0000BC0372D3E7FA51450F474FE0AC072FCA9
:1004C00008C0372D3E7E05C0BA2C372D03C0BA2C8C
:1004D00001C0B52C34FF0DC0FE01EA0DF11D808175
:1004E000803311F4397E09C032FF06C0B394B3944F
:1004F00004C0832F867809F0B39433FD13C030FF16
:1005000006C05A2CB31418F4530C5B18B32CB31454
:1005100068F4B70180E290E03C870E944704B394FE
:100520003C85F5CFB31410F43B1801C0312C34FFD7
:1005300012C0B70180E390E03C870E9447043C85ED
:1005400032FF17C031FD03C088E790E002C088E5A4
:1005500090E0B7010CC0832F867859F031FF02C0BC
:100560008BE201C080E237FD8DE2B70190E00E948E
:100570004704A51438F4B70180E390E00E944704D3
:100580005A94F7CFAA94F401EA0DF11D8081B701C6
:1005900090E00E944704A110F5CF332009F451CE1A
:1005A000B70180E290E00E9447043A94F6CFF70149
:1005B0008681978102C08FEF9FEF2C96E2E10C9429
:1005C000F6040F931F93CF93DF93869F8001879F3D
:1005D000100D969F100D1124C8010E94FD02EC0120
:1005E000009729F0A80160E070E00E943504CE0178
:1005F000DF91CF911F910F910895CF93DF938230B8
:10060000910510F482E090E0E091453EF091463E85
:1006100020E030E0C0E0D0E0309711F1408151811E
:1006200048175907C0F04817590761F48281938130
:10063000209719F08A839B832BC08093453E90932B
:10064000463E26C02115310519F04217530718F40C
:100650009A01BE01DF01EF010280F381E02DDCCFC2
:100660002115310509F1281B390B2430310590F48F
:1006700012968D919C9113976115710521F0FB01E4
:100680008283938304C08093453E9093463EFD0150
:10069000329644C0FD01E20FF31F819391932250E3
:1006A00031092D933C933AC02091433E3091443E12
:1006B000232B41F42091023E3091033E2093433E90
:1006C0003093443E2091003E3091013E211531058A
:1006D00041F42DB73EB74091043E5091053E241B96
:1006E000350BE091433EF091443EE217F307A0F44E
:1006F0002E1B3F0B2817390778F0AC014E5F5F4F78
:100700002417350748F04E0F5F1F4093433E509328
:10071000443E8193919302C0E0E0F0E0CF01DF918D
:10072000CF9108950F931F93CF93DF93009709F410
:100730008CC0FC013297128213820091453E1091C9
:10074000463E0115110581F420813181820F931FEE
:100750002091433E3091443E2817390779F5E093C4
:10076000433EF093443E71C0D80140E050E0AE17E4
:10077000BF0750F412962D913C911397AD012115AE
:10078000310509F1D901F3CF9D01DA0122833383C9
:1007900060817181860F971F8217930769F4EC01BE
:1007A00028813981260F371F2E5F3F4F20833183E9
:1007B0008A819B8182839383452B29F4E093453E74
:1007C000F093463E42C01296ED93FC931397ED01D1
:1007D000499159919E01240F351FE217F30771F4D7
:1007E00080819181840F951F02968D939C93119720
:1007F0008281938112968D939C931397E0E0F0E0B1
:10080000D80112968D919C911397009719F0F801D9
:100810008C01F6CF8D919C9198012E5F3F4F820FF6
:10082000931F2091433E3091443E2817390769F4C5
:10083000309729F41092453E1092463E02C0128233
:1008400013820093433E1093443EDF91CF911F915A
:100850000F910895FC010590615070400110D8F788
:10086000809590958E0F9F1F0895DC0101C06D93B8
:1008700041505040E0F70895FC01615070400190F4
:100880000110D8F7809590958E0F9F1F08950F93B4
:100890001F93CF93DF93FB01238121FD03C08FEFD3
:1008A0009FEF28C022FF16C04681578124813581E1
:1008B0004217530744F4A081B1819D012F5F3F4F40
:1008C000208331838C93268137812F5F3F4F26838E
:1008D000378310C0EB01092F182F0084F185E02D1C
:1008E0000995892BE1F68E819F8101968E839F83E6
:1008F000812F902FDF91CF911F910F910895FA01D1
:10090000AA27283051F1203181F1E8946F936E7F4E
:100910006E5F7F4F8F4F9F4FAF4FB1E03ED0B4E03F
:100920003CD0670F781F891F9A1FA11D680F791F80
:100930008A1F911DA11D6A0F711D811D911DA11D91
:1009400020D009F468943F912AE0269F11243019A1
:10095000305D3193DEF6CF010895462F4770405D3C
:100960004193B3E00FD0C9F7F6CF462F4F70405DEB
:100970004A3318F0495D31FD4052419302D0A9F746
:10098000EACFB4E0A6959795879577956795BA9540
:10099000C9F700976105710508959B01AC010A2E06
:1009A00006945795479537952795BA95C9F7620FDD
:1009B000731F841F951FA01D08952F923F924F9281
:1009C0005F926F927F928F929F92AF92BF92CF92DF
:1009D000DF92EF92FF920F931F93CF93DF93CDB7E8
:1009E000DEB7CA1BDB0BCDBFDEBF09942A8839886E
:1009F00048885F846E847D848C849B84AA84B984B7
:100A0000C884DF80EE80FD800C811B81AA81B981C2
:100A1000CE0FD11DCDBFDEBFED010895F894FFCFFD
:100A20000000473E20004C6967687420696E746559
:100A30006E736974792069732063757272656E7460
:100A40006C79202564206272696768746E657373BF
:0C0A500020706F696E7473210D0A0000A5
:00000001FF
